:020000040000FA
:1000000083160F308500003086002C2028201A200F
:1000100011200B20062810308D071D20831286002A
:1000200008001D200E080C02031D172819288D0A30
:100030001128080000308D00080083120D08890087
:100040008316081408182228831208088E00080056
:10005000831205088C0008008312003089000030EC
:100060008800D0200130890001308800D020023083
:10007000890002308800D0200330890003308800D6
:10008000D0200430890004308800D0200530890059
:1000900005308800D0200630890006308800D02046
:1000A0000730890007308800D020083089000830E8
:1000B0008800D0200930890009308800D0200A301B
:1000C00089000A308800D0200B3089000B3088006E
:1000D000D0200C3089000C308800D0200D308900F1
:1000E0000D308800D0200E3089000E308800D020DE
:1000F0000F3089000F308800D02010308900FC308C
:100100008800D0201130890060308800D020123063
:100110008900DA308800D02013308900F23088005E
:10012000D0201430890066308800D0201530890036
:10013000B6308800D02016308900BE308800D0202C
:1001400017308900E0308800D02018308900FE3058
:100150008800D02019308900F6308800D0201A306D
:100160008900FD308800D0201B3089006130880074
:10017000D0201C308900DB308800D0201D30890061
:10018000F3308800D0201E30890067308800D020EE
:100190001F308900B7308800D0208316081108006E
:1001A0008316081555308900AA30890088148818EC
:0801B000D72808128312080091
:02400E00F13F80
:00000001FF
